BL51 BANKED LINKER/LOCATER V6.22                                                        08/10/2021  11:53:36  PAGE 1


BL51 BANKED LINKER/LOCATER V6.22, INVOKED BY:
D:\PROGRAM FILES\KEIL_C5\C51\BIN\BL51.EXE ..\output\usart.obj, ..\output\stc_it.obj, ..\output\iic.obj, ..\output\main.o
>> bj TO ..\output\c51_iic PRINT (..\lis\c51_iic.m51) RAMSIZE (256)


MEMORY MODEL: SMALL


INPUT MODULES INCLUDED:
  ..\output\usart.obj (USART)
  ..\output\stc_it.obj (STC_IT)
  ..\output\iic.obj (IIC)
  ..\output\main.obj (MAIN)
  D:\PROGRAM FILES\KEIL_C5\C51\LIB\C51S.LIB (?C_STARTUP)
  D:\PROGRAM FILES\KEIL_C5\C51\LIB\C51S.LIB (?C?COPY)
  D:\PROGRAM FILES\KEIL_C5\C51\LIB\C51S.LIB (?C?CLDOPTR)
  D:\PROGRAM FILES\KEIL_C5\C51\LIB\C51S.LIB (?C?CILDOPTR)
  D:\PROGRAM FILES\KEIL_C5\C51\LIB\C51S.LIB (?C?CSTPTR)
  D:\PROGRAM FILES\KEIL_C5\C51\LIB\C51S.LIB (?C?ILDOPTR)
  D:\PROGRAM FILES\KEIL_C5\C51\LIB\C51S.LIB (?C?ISTPTR)
  D:\PROGRAM FILES\KEIL_C5\C51\LIB\C51S.LIB (?C?ULDIV)
  D:\PROGRAM FILES\KEIL_C5\C51\LIB\C51S.LIB (PRINTF)
  D:\PROGRAM FILES\KEIL_C5\C51\LIB\C51S.LIB (?C?MEMSET)
  D:\PROGRAM FILES\KEIL_C5\C51\LIB\C51S.LIB (?C_INIT)
  D:\PROGRAM FILES\KEIL_C5\C51\LIB\C51S.LIB (?C?CLDPTR)
  D:\PROGRAM FILES\KEIL_C5\C51\LIB\C51S.LIB (?C?PLDIIDATA)
  D:\PROGRAM FILES\KEIL_C5\C51\LIB\C51S.LIB (?C?CCASE)


LINK MAP OF MODULE:  ..\output\c51_iic (USART)


            TYPE    BASE      LENGTH    RELOCATION   SEGMENT NAME
            -----------------------------------------------------

            * * * * * * *   D A T A   M E M O R Y   * * * * * * *
            REG     0000H     0008H     ABSOLUTE     "REG BANK 0"
            DATA    0008H     0016H     UNIT         _DATA_GROUP_
            DATA    001EH     0002H     UNIT         ?DT?USART
            BIT     0020H.0   0001H.1   UNIT         _BIT_GROUP_
                    0021H.1   0000H.7                *** GAP ***
            DATA    0022H     0013H     UNIT         ?DT?_SEND_OUT?USART
            DATA    0035H     0012H     UNIT         ?DT?_SEND_3OUT?USART
            DATA    0047H     0006H     UNIT         ?DT?_SINGLE_READI2C?IIC
            DATA    004DH     0005H     UNIT         ?DT?STC_IT
            DATA    0052H     0004H     UNIT         ?DT?_USART_SEND?USART
            IDATA   0056H     0001H     UNIT         ?STACK

            * * * * * * *   C O D E   M E M O R Y   * * * * * * *
            CODE    0000H     0003H     ABSOLUTE     
            CODE    0003H     000EH     UNIT         ?PR?_PUTCHAR?MAIN
            CODE    0011H     0002H     UNIT         ?CO?IIC
            CODE    0013H     0003H     ABSOLUTE     
            CODE    0016H     000DH     UNIT         ?CO?USART
            CODE    0023H     0003H     ABSOLUTE     
            CODE    0026H     035CH     UNIT         ?PR?PRINTF?PRINTF
            CODE    0382H     0308H     UNIT         ?C?LIB_CODE
            CODE    068AH     00A2H     UNIT         ?PR?_SEND_OUT?USART
BL51 BANKED LINKER/LOCATER V6.22                                                      08/10/2021  11:53:36  PAGE 2


            CODE    072CH     008CH     UNIT         ?C_C51STARTUP
            CODE    07B8H     0080H     UNIT         ?PR?_SINGLE_READI2C?IIC
            CODE    0838H     006CH     UNIT         ?PR?_SEND_3OUT?USART
            CODE    08A4H     0063H     UNIT         ?PR?_REQUESTRANGE?IIC
            CODE    0907H     005CH     UNIT         ?PR?USART_IRQHANDLER?STC_IT
            CODE    0963H     0053H     UNIT         ?PR?_USART_SEND?USART
            CODE    09B6H     003EH     UNIT         ?PR?_SINGLE_WRITEI2C_BYTE?IIC
            CODE    09F4H     0037H     UNIT         ?PR?_TAKERANGEREADING?IIC
            CODE    0A2BH     0036H     UNIT         ?PR?MAIN?MAIN
            CODE    0A61H     002EH     UNIT         ?PR?_USART_INT?USART
            CODE    0A8FH     0027H     UNIT         ?PR?I2C_RECVBYTE?IIC
            CODE    0AB6H     0025H     UNIT         ?PR?I2C_START?IIC
            CODE    0ADBH     0025H     UNIT         ?PR?_I2C_SENDBYTE?IIC
            CODE    0B00H     0020H     UNIT         ?PR?I2C_WAITACK?IIC
            CODE    0B20H     0015H     UNIT         ?PR?_I2C_SENDACK?IIC
            CODE    0B35H     0012H     UNIT         ?C_INITSEG
            CODE    0B47H     0011H     UNIT         ?PR?I2C_STOP?IIC
            CODE    0B58H     000DH     UNIT         ?CO?MAIN
            CODE    0B65H     000BH     UNIT         ?PR?_DELAY?MAIN
            CODE    0B70H     000AH     UNIT         ?PR?_USART_SEND_BYTE?USART
            CODE    0B7AH     0003H     UNIT         ?PR?_DELAY_1US?IIC
            CODE    0B7DH     0001H     UNIT         ?PR?EXTI1_IRQHANDLER?STC_IT



OVERLAY MAP OF MODULE:   ..\output\c51_iic (USART)


SEGMENT                                  BIT_GROUP          DATA_GROUP 
  +--> CALLED SEGMENT                 START    LENGTH     START    LENGTH
-------------------------------------------------------------------------
?C_C51STARTUP                         -----    -----      -----    -----
  +--> ?PR?MAIN?MAIN
  +--> ?C_INITSEG

?PR?MAIN?MAIN                         -----    -----      0008H    0002H
  +--> ?PR?_USART_INT?USART
  +--> ?PR?_REQUESTRANGE?IIC
  +--> ?PR?_TAKERANGEREADING?IIC
  +--> ?CO?MAIN
  +--> ?PR?PRINTF?PRINTF
  +--> ?PR?_DELAY?MAIN

?PR?_USART_INT?USART                  -----    -----      000AH    0004H

?PR?_REQUESTRANGE?IIC                 -----    -----      000AH    0006H
  +--> ?CO?IIC
  +--> ?PR?I2C_START?IIC
  +--> ?PR?_I2C_SENDBYTE?IIC
  +--> ?PR?I2C_WAITACK?IIC
  +--> ?PR?I2C_STOP?IIC
  +--> ?PR?_DELAY_1US?IIC
  +--> ?PR?I2C_RECVBYTE?IIC
  +--> ?PR?_I2C_SENDACK?IIC

?PR?I2C_START?IIC                     -----    -----      -----    -----
  +--> ?PR?_DELAY_1US?IIC
BL51 BANKED LINKER/LOCATER V6.22                                                      08/10/2021  11:53:36  PAGE 3



?PR?_DELAY_1US?IIC                    -----    -----      0010H    0001H

?PR?_I2C_SENDBYTE?IIC                 -----    -----      -----    -----
  +--> ?PR?_DELAY_1US?IIC

?PR?I2C_WAITACK?IIC                   -----    -----      -----    -----
  +--> ?PR?_DELAY_1US?IIC

?PR?I2C_STOP?IIC                      -----    -----      -----    -----
  +--> ?PR?_DELAY_1US?IIC

?PR?I2C_RECVBYTE?IIC                  -----    -----      -----    -----
  +--> ?PR?_DELAY_1US?IIC

?PR?_I2C_SENDACK?IIC                  -----    -----      -----    -----
  +--> ?PR?_DELAY_1US?IIC

?PR?_TAKERANGEREADING?IIC             -----    -----      -----    -----
  +--> ?PR?_DELAY_1US?IIC
  +--> ?PR?I2C_START?IIC
  +--> ?PR?_I2C_SENDBYTE?IIC
  +--> ?PR?I2C_WAITACK?IIC
  +--> ?PR?I2C_STOP?IIC

?PR?PRINTF?PRINTF                     0020H.0  0001H.1    000AH    0014H
  +--> ?PR?_PUTCHAR?MAIN



SYMBOL TABLE OF MODULE:  ..\output\c51_iic (USART)

  VALUE           TYPE          NAME
  ----------------------------------

  -------         MODULE        USART
  C:0000H         SYMBOL        _ICE_DUMMY_
  D:0080H         PUBLIC        P0
  D:0090H         PUBLIC        P1
  D:00B0H         PUBLIC        P3
  D:00A8H         PUBLIC        IE
  D:00B8H         PUBLIC        IP
  C:0838H         PUBLIC        _send_3out
  C:0A61H         PUBLIC        _Usart_Int
  D:0099H         PUBLIC        SBUF
  D:0098H         PUBLIC        SCON
  C:0B70H         PUBLIC        _USART_send_byte
  D:0089H         PUBLIC        TMOD
  D:0088H         PUBLIC        TCON
  C:0016H         SYMBOL        _?ix1000
  D:008DH         PUBLIC        TH1
  D:008BH         PUBLIC        TL1
  C:068AH         PUBLIC        _send_out
  D:001EH         PUBLIC        send_ok
  D:00C8H         PUBLIC        T2CON
  D:001FH         PUBLIC        Calibration
  D:00D0H         PUBLIC        PSW
BL51 BANKED LINKER/LOCATER V6.22                                                      08/10/2021  11:53:36  PAGE 4


  C:0963H         PUBLIC        _USART_Send
  -------         PROC          _USART_INT
  D:000AH         SYMBOL        BaudRatePrescaler
  C:0A61H         LINE#         4
  C:0A69H         LINE#         5
  C:0A69H         LINE#         6
  C:0A6CH         LINE#         7
  C:0A6FH         LINE#         9
  C:0A86H         LINE#         10
  C:0A88H         LINE#         11
  C:0A8BH         LINE#         12
  C:0A8EH         LINE#         13
  -------         ENDPROC       _USART_INT
  -------         PROC          _USART_SEND_BYTE
  D:0007H         SYMBOL        Tx_data
  C:0B70H         LINE#         16
  C:0B70H         LINE#         17
  C:0B70H         LINE#         18
  C:0B74H         LINE#         19
  C:0B76H         LINE#         20
  C:0B79H         LINE#         21
  -------         ENDPROC       _USART_SEND_BYTE
  -------         PROC          _USART_SEND
  D:0052H         SYMBOL        Buffer
  D:0005H         SYMBOL        Length
  -------         DO            
  D:0055H         SYMBOL        i
  -------         ENDDO         
  C:0963H         LINE#         23
  C:0969H         LINE#         24
  C:0969H         LINE#         25
  C:096CH         LINE#         26
  C:0972H         LINE#         27
  C:0972H         LINE#         28
  C:097BH         LINE#         29
  C:099DH         LINE#         30
  C:09B3H         LINE#         31
  C:09B5H         LINE#         32
  -------         ENDPROC       _USART_SEND
  -------         PROC          _SEND_3OUT
  D:0035H         SYMBOL        Data
  D:0038H         SYMBOL        length
  D:0039H         SYMBOL        send
  -------         DO            
  D:003AH         SYMBOL        TX_DATA
  D:0007H         SYMBOL        i
  D:0006H         SYMBOL        k
  -------         ENDDO         
  C:0838H         LINE#         33
  C:0840H         LINE#         34
  C:0840H         LINE#         35
  C:0855H         LINE#         36
  C:085BH         LINE#         37
  C:0863H         LINE#         38
  C:086BH         LINE#         39
  C:0873H         LINE#         40
  C:087BH         LINE#         41
BL51 BANKED LINKER/LOCATER V6.22                                                      08/10/2021  11:53:36  PAGE 5


  C:087BH         LINE#         42
  C:0893H         LINE#         43
  C:0896H         LINE#         44
  -------         ENDPROC       _SEND_3OUT
  -------         PROC          _SEND_OUT
  D:0022H         SYMBOL        Data
  D:0025H         SYMBOL        length
  D:0026H         SYMBOL        send
  -------         DO            
  D:0027H         SYMBOL        TX_DATA
  D:0034H         SYMBOL        i
  D:0005H         SYMBOL        k
  -------         ENDDO         
  C:068AH         LINE#         47
  C:0692H         LINE#         48
  C:0692H         LINE#         49
  C:0696H         LINE#         50
  C:06ACH         LINE#         51
  C:06B6H         LINE#         52
  C:06C0H         LINE#         53
  C:06CAH         LINE#         54
  C:06D9H         LINE#         55
  C:06E1H         LINE#         56
  C:06E1H         LINE#         57
  C:0701H         LINE#         58
  C:0719H         LINE#         59
  C:071CH         LINE#         60
  -------         ENDPROC       _SEND_OUT
  -------         ENDMOD        USART

  -------         MODULE        STC_IT
  C:0000H         SYMBOL        _ICE_DUMMY_
  D:0080H         PUBLIC        P0
  D:0090H         PUBLIC        P1
  D:00B0H         PUBLIC        P3
  D:00A8H         PUBLIC        IE
  D:00B8H         PUBLIC        IP
  B:0098H.0       PUBLIC        RI
  B:0098H.1       PUBLIC        TI
  D:0051H         PUBLIC        stata
  C:0907H         PUBLIC        USART_IRQHandler
  D:0099H         PUBLIC        SBUF
  D:0098H         PUBLIC        SCON
  D:0088H         PUBLIC        TCON
  D:00C8H         PUBLIC        T2CON
  D:00D0H         PUBLIC        PSW
  C:0B7DH         PUBLIC        EXTI1_IRQHandler
  -------         PROC          EXTI1_IRQHANDLER
  C:0B7DH         LINE#         6
  C:0B7DH         LINE#         8
  -------         ENDPROC       EXTI1_IRQHANDLER
  -------         PROC          USART_IRQHANDLER
  -------         DO            
  D:004DH         SYMBOL        i
  D:004EH         SYMBOL        rebuf
  D:0007H         SYMBOL        sum
  -------         ENDDO         
BL51 BANKED LINKER/LOCATER V6.22                                                      08/10/2021  11:53:36  PAGE 6


  C:0907H         LINE#         10
  C:0914H         LINE#         13
  C:0915H         LINE#         14
  C:0918H         LINE#         15
  C:0918H         LINE#         16
  C:091AH         LINE#         17
  C:091CH         LINE#         18
  C:091CH         LINE#         19
  C:091FH         LINE#         20
  C:091FH         LINE#         21
  C:0929H         LINE#         22
  C:092BH         LINE#         23
  C:0936H         LINE#         24
  C:0939H         LINE#         25
  C:093EH         LINE#         26
  C:093EH         LINE#         27
  C:0942H         LINE#         28
  C:0945H         LINE#         29
  C:0945H         LINE#         30
  C:094AH         LINE#         31
  C:094AH         LINE#         32
  C:094DH         LINE#         34
  C:094DH         LINE#         35
  C:0952H         LINE#         36
  C:0952H         LINE#         37
  C:0955H         LINE#         39
  C:0955H         LINE#         40
  C:0955H         LINE#         41
  C:0958H         LINE#         42
  C:0958H         LINE#         44
  C:0958H         LINE#         46
  -------         ENDPROC       USART_IRQHANDLER
  -------         ENDMOD        STC_IT

  -------         MODULE        IIC
  C:0000H         SYMBOL        _ICE_DUMMY_
  C:08A4H         PUBLIC        _requestRange
  D:0090H         PUBLIC        P1
  D:00B0H         PUBLIC        P3
  C:07B8H         PUBLIC        _Single_ReadI2C
  C:0B7AH         PUBLIC        _delay_1us
  D:00A8H         PUBLIC        IE
  D:00B8H         PUBLIC        IP
  C:09B6H         PUBLIC        _Single_WriteI2C_byte
  C:0AB6H         PUBLIC        I2C_Start
  D:0098H         PUBLIC        SCON
  D:0088H         PUBLIC        TCON
  C:0ADBH         PUBLIC        _I2C_SendByte
  C:0011H         SYMBOL        _?ix1000
  C:0B00H         PUBLIC        I2C_WaitAck
  C:0B47H         PUBLIC        I2C_Stop
  C:0A8FH         PUBLIC        I2C_RecvByte
  C:09F4H         PUBLIC        _takeRangeReading
  B:00B0H.7       PUBLIC        SDA
  B:00B0H.6       PUBLIC        SCL
  D:00C8H         PUBLIC        T2CON
  D:00D0H         PUBLIC        PSW
BL51 BANKED LINKER/LOCATER V6.22                                                      08/10/2021  11:53:36  PAGE 7


  C:0B20H         PUBLIC        _I2C_SendACK
  -------         PROC          _DELAY_1US
  D:0010H         SYMBOL        x
  C:0B7AH         LINE#         2
  C:0B7CH         LINE#         3
  C:0B7CH         LINE#         5
  -------         ENDPROC       _DELAY_1US
  -------         PROC          I2C_START
  C:0AB6H         LINE#         11
  C:0AB6H         LINE#         12
  C:0AB6H         LINE#         13
  C:0AB8H         LINE#         14
  C:0ABDH         LINE#         15
  C:0ABFH         LINE#         16
  C:0AC2H         LINE#         17
  C:0AC7H         LINE#         18
  C:0AC9H         LINE#         19
  C:0ACEH         LINE#         20
  C:0AD3H         LINE#         21
  C:0AD5H         LINE#         22
  C:0ADAH         LINE#         23
  C:0ADAH         LINE#         24
  -------         ENDPROC       I2C_START
  -------         PROC          I2C_STOP
  C:0B47H         LINE#         31
  C:0B47H         LINE#         32
  C:0B47H         LINE#         33
  C:0B49H         LINE#         34
  C:0B4BH         LINE#         35
  C:0B50H         LINE#         36
  C:0B52H         LINE#         37
  C:0B55H         LINE#         38
  C:0B57H         LINE#         39
  -------         ENDPROC       I2C_STOP
  -------         PROC          _I2C_SENDACK
  D:0007H         SYMBOL        i
  C:0B20H         LINE#         48
  C:0B20H         LINE#         49
  C:0B20H         LINE#         50
  C:0B23H         LINE#         51
  C:0B27H         LINE#         53
  C:0B29H         LINE#         54
  C:0B2BH         LINE#         55
  C:0B30H         LINE#         56
  C:0B32H         LINE#         57
  -------         ENDPROC       _I2C_SENDACK
  -------         PROC          I2C_WAITACK
  -------         DO            
  D:0007H         SYMBOL        i
  -------         ENDDO         
  C:0B00H         LINE#         65
  C:0B00H         LINE#         66
  C:0B00H         LINE#         67
  C:0B02H         LINE#         68
  C:0B04H         LINE#         69
  C:0B06H         LINE#         70
  C:0B09H         LINE#         71
BL51 BANKED LINKER/LOCATER V6.22                                                      08/10/2021  11:53:36  PAGE 8


  C:0B09H         LINE#         72
  C:0B0AH         LINE#         73
  C:0B0DH         LINE#         74
  C:0B0DH         LINE#         76
  C:0B10H         LINE#         77
  C:0B10H         LINE#         78
  C:0B12H         LINE#         79
  C:0B15H         LINE#         80
  C:0B15H         LINE#         81
  C:0B1AH         LINE#         82
  C:0B1CH         LINE#         83
  C:0B1FH         LINE#         84
  C:0B1FH         LINE#         85
  -------         ENDPROC       I2C_WAITACK
  -------         PROC          _I2C_SENDBYTE
  D:0006H         SYMBOL        dat
  -------         DO            
  D:0005H         SYMBOL        i
  -------         ENDDO         
  C:0ADBH         LINE#         92
  C:0ADDH         LINE#         93
  C:0ADDH         LINE#         95
  C:0ADFH         LINE#         96
  C:0AE1H         LINE#         97
  C:0AE1H         LINE#         98
  C:0AE5H         LINE#         99
  C:0AE9H         LINE#         101
  C:0AEBH         LINE#         102
  C:0AEDH         LINE#         103
  C:0AF2H         LINE#         104
  C:0AF4H         LINE#         105
  C:0AF7H         LINE#         106
  C:0AFBH         LINE#         107
  C:0AFFH         LINE#         108
  -------         ENDPROC       _I2C_SENDBYTE
  -------         PROC          I2C_RECVBYTE
  -------         DO            
  D:0005H         SYMBOL        i
  D:0006H         SYMBOL        dat
  -------         ENDDO         
  C:0A8FH         LINE#         112
  C:0A8FH         LINE#         113
  C:0A8FH         LINE#         115
  C:0A91H         LINE#         116
  C:0A93H         LINE#         117
  C:0A98H         LINE#         118
  C:0A99H         LINE#         119
  C:0A99H         LINE#         120
  C:0A9DH         LINE#         122
  C:0A9FH         LINE#         124
  C:0AA2H         LINE#         125
  C:0AA5H         LINE#         126
  C:0AAAH         LINE#         127
  C:0AACH         LINE#         128
  C:0AAFH         LINE#         129
  C:0AB3H         LINE#         130
  C:0AB5H         LINE#         131
BL51 BANKED LINKER/LOCATER V6.22                                                      08/10/2021  11:53:36  PAGE 9


  -------         ENDPROC       I2C_RECVBYTE
  -------         PROC          _SINGLE_WRITEI2C_BYTE
  D:0006H         SYMBOL        Slave_Address
  D:0003H         SYMBOL        REG_Address
  D:0004H         SYMBOL        datas
  C:09B6H         LINE#         135
  C:09BCH         LINE#         136
  C:09BCH         LINE#         137
  C:09C2H         LINE#         138
  C:09C4H         LINE#         140
  C:09C9H         LINE#         141
  C:09D1H         LINE#         143
  C:09D6H         LINE#         144
  C:09DEH         LINE#         146
  C:09E3H         LINE#         147
  C:09EEH         LINE#         149
  C:09F1H         LINE#         151
  C:09F3H         LINE#         152
  -------         ENDPROC       _SINGLE_WRITEI2C_BYTE
  -------         PROC          _SINGLE_READI2C
  D:0004H         SYMBOL        Slave_Address
  D:0048H         SYMBOL        REG_Address
  D:0049H         SYMBOL        REG_data
  D:004CH         SYMBOL        length
  C:07B8H         LINE#         156
  C:07C2H         LINE#         157
  C:07C2H         LINE#         158
  C:07C8H         LINE#         159
  C:07CAH         LINE#         161
  C:07CFH         LINE#         162
  C:07D7H         LINE#         164
  C:07DCH         LINE#         165
  C:07E4H         LINE#         167
  C:07EAH         LINE#         168
  C:07ECH         LINE#         170
  C:07F2H         LINE#         171
  C:07FDH         LINE#         173
  C:0802H         LINE#         174
  C:0802H         LINE#         175
  C:0817H         LINE#         176
  C:081CH         LINE#         177
  C:081EH         LINE#         178
  C:0820H         LINE#         179
  C:082DH         LINE#         180
  C:0832H         LINE#         181
  C:0835H         LINE#         182
  C:0837H         LINE#         183
  -------         ENDPROC       _SINGLE_READI2C
  -------         PROC          _TAKERANGEREADING
  D:0006H         SYMBOL        Slave_Address
  C:09F4H         LINE#         184
  C:09F6H         LINE#         185
  C:09FBH         LINE#         186
  C:0A01H         LINE#         187
  C:0A03H         LINE#         189
  C:0A08H         LINE#         190
  C:0A10H         LINE#         191
BL51 BANKED LINKER/LOCATER V6.22                                                      08/10/2021  11:53:36  PAGE 10


  C:0A15H         LINE#         192
  C:0A1AH         LINE#         193
  C:0A25H         LINE#         196
  C:0A28H         LINE#         197
  C:0A2AH         LINE#         198
  -------         ENDPROC       _TAKERANGEREADING
  -------         PROC          _REQUESTRANGE
  D:000AH         SYMBOL        Slave_Address
  D:000BH         SYMBOL        distance
  -------         DO            
  D:000EH         SYMBOL        REG_data
  -------         ENDDO         
  C:08A4H         LINE#         199
  C:08ACH         LINE#         200
  C:08BFH         LINE#         203
  C:08C5H         LINE#         204
  C:08C7H         LINE#         206
  C:08CCH         LINE#         207
  C:08D7H         LINE#         208
  C:08DCH         LINE#         211
  C:08E1H         LINE#         213
  C:08E6H         LINE#         215
  C:08EBH         LINE#         217
  C:08F0H         LINE#         219
  C:08F3H         LINE#         220
  C:0904H         LINE#         221
  C:0906H         LINE#         222
  -------         ENDPROC       _REQUESTRANGE
  -------         ENDMOD        IIC

  -------         MODULE        MAIN
  C:0000H         SYMBOL        _ICE_DUMMY_
  D:0080H         PUBLIC        P0
  D:0090H         PUBLIC        P1
  D:00B0H         PUBLIC        P3
  D:00A8H         PUBLIC        IE
  C:0B65H         PUBLIC        _delay
  B:00A8H.4       PUBLIC        ES
  D:00B8H         PUBLIC        IP
  B:0098H.1       PUBLIC        TI
  C:0A2BH         PUBLIC        main
  D:0099H         PUBLIC        SBUF
  D:0098H         PUBLIC        SCON
  D:0088H         PUBLIC        TCON
  D:00C8H         PUBLIC        T2CON
  D:00D0H         PUBLIC        PSW
  C:0003H         PUBLIC        _putchar
  -------         PROC          _PUTCHAR
  D:0007H         SYMBOL        c
  C:0003H         LINE#         20
  C:0003H         LINE#         21
  C:0003H         LINE#         22
  C:0005H         LINE#         23
  C:0007H         LINE#         24
  C:000AH         LINE#         25
  C:000CH         LINE#         26
  C:000EH         LINE#         27
BL51 BANKED LINKER/LOCATER V6.22                                                      08/10/2021  11:53:36  PAGE 11


  C:0010H         LINE#         28
  -------         ENDPROC       _PUTCHAR
  -------         PROC          _DELAY
  D:0006H         SYMBOL        x
  C:0B65H         LINE#         29
  C:0B65H         LINE#         30
  C:0B65H         LINE#         31
  C:0B6FH         LINE#         32
  -------         ENDPROC       _DELAY
  -------         PROC          MAIN
  -------         DO            
  D:0008H         SYMBOL        distance
  -------         ENDDO         
  C:0A2BH         LINE#         33
  C:0A2BH         LINE#         34
  C:0A2BH         LINE#         35
  C:0A30H         LINE#         36
  C:0A39H         LINE#         37
  C:0A39H         LINE#         38
  C:0A39H         LINE#         40
  C:0A44H         LINE#         41
  C:0A49H         LINE#         43
  C:0A58H         LINE#         44
  C:0A5FH         LINE#         45
  -------         ENDPROC       MAIN
  -------         ENDMOD        MAIN

  -------         MODULE        ?C?COPY
  C:0452H         PUBLIC        ?C?COPY
  -------         ENDMOD        ?C?COPY

  -------         MODULE        ?C?CLDOPTR
  C:0478H         PUBLIC        ?C?CLDOPTR
  -------         ENDMOD        ?C?CLDOPTR

  -------         MODULE        ?C?CILDOPTR
  C:04A5H         PUBLIC        ?C?CILDOPTR
  -------         ENDMOD        ?C?CILDOPTR

  -------         MODULE        ?C?CSTPTR
  C:04D8H         PUBLIC        ?C?CSTPTR
  -------         ENDMOD        ?C?CSTPTR

  -------         MODULE        ?C?ILDOPTR
  C:04EAH         PUBLIC        ?C?ILDOPTR
  -------         ENDMOD        ?C?ILDOPTR

  -------         MODULE        ?C?ISTPTR
  C:0522H         PUBLIC        ?C?ISTPTR
  -------         ENDMOD        ?C?ISTPTR

  -------         MODULE        ?C?ULDIV
  C:057DH         PUBLIC        ?C?ULDIV
  -------         ENDMOD        ?C?ULDIV

  -------         MODULE        PRINTF
  D:000AH         PUBLIC        ?_PRINTF517?BYTE
BL51 BANKED LINKER/LOCATER V6.22                                                      08/10/2021  11:53:36  PAGE 12


  D:000AH         PUBLIC        ?_PRINTF?BYTE
  D:000AH         PUBLIC        ?_SPRINTF517?BYTE
  D:000AH         PUBLIC        ?_SPRINTF?BYTE
  C:0088H         PUBLIC        _PRINTF
  C:0088H         PUBLIC        _PRINTF517
  C:0082H         PUBLIC        _SPRINTF
  C:0082H         PUBLIC        _SPRINTF517
  -------         ENDMOD        PRINTF

  -------         MODULE        ?C?MEMSET
  C:060FH         PUBLIC        ?C?MEMSET
  -------         ENDMOD        ?C?MEMSET

  -------         MODULE        ?C?CLDPTR
  C:063BH         PUBLIC        ?C?CLDPTR
  -------         ENDMOD        ?C?CLDPTR

  -------         MODULE        ?C?PLDIIDATA
  C:0654H         PUBLIC        ?C?PLDIIDATA
  -------         ENDMOD        ?C?PLDIIDATA

  -------         MODULE        ?C?CCASE
  C:0664H         PUBLIC        ?C?CCASE
  -------         ENDMOD        ?C?CCASE

*** WARNING L16: UNCALLED SEGMENT, IGNORED FOR OVERLAY PROCESS
    SEGMENT: ?PR?_SEND_3OUT?USART

*** WARNING L16: UNCALLED SEGMENT, IGNORED FOR OVERLAY PROCESS
    SEGMENT: ?PR?_SEND_OUT?USART

*** WARNING L16: UNCALLED SEGMENT, IGNORED FOR OVERLAY PROCESS
    SEGMENT: ?PR?_SINGLE_WRITEI2C_BYTE?IIC

*** WARNING L16: UNCALLED SEGMENT, IGNORED FOR OVERLAY PROCESS
    SEGMENT: ?PR?_SINGLE_READI2C?IIC

Program Size: data=86.1 xdata=0 code=2942
LINK/LOCATE RUN COMPLETE.  4 WARNING(S),  0 ERROR(S)
